:020000040000FA
:04000000640023284D
:080008000F398A018207CE2D99
:10001000D82DE12DEB2DF52DFF2D092E132E1D2EA4
:10002000272E1D2E1D2E1D2E1D2E1D2E1D2E8A012E
:100030008207562A622A6E2A7A2A862A922A9E2ABB
:10004000AA2AB62AC22A850107309F00003065001F
:1000500086010130660003306200353090008F0168
:100060008E010C100022A001A101A301A2011A21FE
:10007000AC016400061839288E018F010C10640051
:100080000C183328061C3F2864000C183328061867
:1000900044281010B2010F08B3000E08B4008E01FE
:1000A0008F010C10101494205D203F283008BC00F4
:1000B0003108BB00852002213F282C08003A031D8F
:1000C0006428BB01BC01BD013108BB07031C6C28BF
:1000D0000310BC0A0318BD0A3008BC070318BD0A88
:1000E000AC0A2C08213A031D0800AC01BD0CBC0C65
:1000F000BB0CBD0CBC0CBB0CBD0CBC0CBB0CBD0CC0
:10010000BC0CBB0CBD0CBC0CBB0CDF2040080F3979
:10011000A000400E0F39A1003F080F39A2003F0E8A
:100120000F39A3001A2108003408003A031D9F2844
:100130003308003A031D9F28B101B001003400309C
:10014000D820B8000130D820B9000230D820BA0039
:100150001830C100AF01B001B101B501B601B7015E
:100160000310BA0DB90DB80DB70DB60DB50D3208A7
:100170003502031DC12833083602031DC128340887
:100180003702031CD2283408B702031CB603360812
:10019000FF3A0319B5033308B602031CB50332084E
:1001A000B5020314B10DB00DAF0DC10BB02808009E
:1001B000831603139B001C141A08831208000310F3
:1001C0001030C100BE01BF01C001BB0DBC0DC00D90
:1001D000BF0DBE0DC10BED28080040308400F72094
:1001E0003F308400F7203E308400F720E5280330BC
:1001F0000007C200C219800030300007C200C21BD5
:1002000080000800FF30AD00AE001521152115213A
:1002100015211521AE0B05290800FF30AD00AE00F9
:1002200015211521AE0B10290800AD0B152908006A
:10023000640018298330A9004030AA002208172042
:100240009830A9004030AA0021081720AD30A9003D
:100250004030AA0020081720C230A9004030AA0070
:0602600003011720080055
:10040000422286161C2221301822C53018221330B1
:1004100018222030182209302E22192208301822E2
:100420000C30182208000301A40086162022003494
:10043000A40086122022003406124222061600343E
:100440000830A8008613A41B0617A41F0613640017
:1004500086170000A40DA80B222A0034A40006135E
:100460000630A7005430A5000830A6008616861373
:10047000640000008617A60B372AA50B342AA70BA9
:10048000322A003464000730A70064003230A5002F
:100490006400FA30A600A60B4B2AA50B482AA70B2E
:1004A000452A0034290818222A08182A5222122321
:1004B000AA0A5222F522AA0A5222CE22AA0A5222BD
:1004C000812308005222E122AA0A5222EB22AA0A20
:1004D00052220823AA0A52228E2408005222A6235E
:1004E000AA0A5222CA23AA0A5222ED23AA0A522297
:1004F000102408005222A623AA0A5222CA23AA0ABA
:1005000052223424AA0A52225724080052227B2461
:10051000AA0A52223723AA0A52223424AA0A5222B1
:100520008E24080052229824AA0A5222BC24AA0A25
:1005300052223424AA0A5222572408005222982414
:10054000AA0A5222BC24AA0A52225C23AA0A5222D4
:100550008123080052221223AA0A5222F522AA0A53
:1005600052220823AA0A52228E2408005222122361
:10057000AA0A52223723AA0A52225C23AA0A52222A
:100580008123080052221223AA0A52223723AA0AE0
:1005900052223424AA0A522257240800FF3014227F
:1005A000FE301422FC301422F83014220A30E024E9
:1005B000F8301422FC301422FE301422FF301422B2
:1005C0000800DF24F0301422F8301422FC3014220A
:1005D000FE3014220800DF241F3014223F30142282
:1005E0007F301422FF3014220800FF3014227F30A5
:1005F00014223F3014221F3014220A30E0241F300E
:1006000014223F3014227F301422FF3014220800BD
:10061000DF24F8301422FC301422FE301422FF3084
:1006200014220800FE301422FD301422FB30142264
:10063000F73014220F3014220F3014220F301422FE
:100640000F3014220F3014220F3014220F301422D6
:100650000F3014220F3014220F301422F7301422DE
:10066000FB301422FD301422FE3014220800FF302B
:1006700014227F301422BF301422DF301422C03005
:100680001422C0301422C0301422C0301422C030D2
:100690001422C0301422C0301422C0301422C030C2
:1006A0001422C0301422DF301422BF3014227F30D5
:1006B0001422FF3014220800FF301422FE301422CE
:1006C000FD301422FB301422033014220330142294
:1006D0000330142203301422033014220330142276
:1006E0000330142203301422033014220330142266
:1006F000FB301422FD301422FE301422FF3014226D
:1007000008007F301422BF301422DF301422EF3073
:100710001422F0301422F0301422F0301422F03081
:100720001422F0301422F0301422F0301422F03071
:100730001422F0301422F0301422EF301422DF3073
:100740001422BF3014227F301422080013220130FB
:10075000142203301422073014220F3014220F30D9
:1007600014220F3014220F3014220F3014220F30B5
:1007700014220F3014220F3014220F3014220F30A5
:100780001422F7301422FB301422FD301422FE30E4
:10079000142208001322132280301422C0301422A5
:1007A000C0301422C0301422C0301422C0301422B1
:1007B000C0301422C0301422C0301422C0301422A1
:1007C000C0301422C0301422DF301422BF30142273
:1007D0007F301422FF3014220800FF301422FE3034
:1007E0001422FD301422FB30142203301422033073
:1007F0001422033014220330142203301422033055
:100800001422033014220330142203301422033044
:100810001422033014220130142213221322080060
:100820007F301422BF301422DF301422EF30142224
:10083000F0301422F0301422F0301422F030142260
:10084000F0301422F0301422F0301422F030142250
:10085000F0301422F0301422E0301422C030142280
:100860008030142213220800132213220130142294
:1008700003301422033014220330142203301422D4
:1008800003301422033014220330142203301422C4
:10089000033014220330142203301422FB301422BC
:1008A000FD301422FE301422FF30142208001322DF
:1008B00080301422C0301422E0301422F030142290
:1008C000F0301422F0301422F0301422F0301422D0
:1008D000F0301422F0301422F0301422F0301422C0
:1008E000F0301422EF301422DF301422BF301422F3
:1008F0007F3014220800FE301422FC301422F8301D
:100900001422F03014220A30E024F0301422F8309F
:100910001422FC301422FE3014220800DF241F3081
:1009200014223F3014227F301422FF30142208009A
:10093000FE301422FD301422FB301422F730142232
:100940000F3014220F3014220F3014220F301422D3
:100950000F3014220F3014220F3014220F301422C3
:100960000F3014220F3014220730142203301422C7
:100970000130142213220800FF3014227F30142289
:10098000BF301422DF301422C0301422C0301422B1
:10099000C0301422C0301422C0301422C0301422BF
:1009A000C0301422C0301422C0301422C0301422AF
:1009B000C0301422803014221322132208000E307B
:1009C000A5001322A50BE12C08005222AC25AA0A8F
:1009D00052229B25080052222125AA0A52222E25A6
:1009E000080052226825AA0A5222792508005222BC
:1009F0006825AA0A52228A25080052224A25AA0AF4
:100A000052225725080052223925AA0A52228A2545
:100A1000080052223925AA0A5222BD250800522276
:100A2000AC25AA0A52222E2508005222AC25AA0A79
:100A30005222BD2508005222AC25AA0A52228A253C
:100A400008001322132213221322303014223030D4
:100A50001422FC301422FC3014220800132213222A
:100A60001322132213221322FF301422FF301422E8
:100A70000800FC301422FC3014220C3014220C30FC
:100A800014220C3014220C3014220C3014220C309E
:100A900014220800FC301422FC30142213221322EA
:100AA00013221322FC301422FC30142208000330DD
:100AB0001422033014220330142203301422033092
:100AC000142203301422FF301422FF3014220800B5
:100AD0000C3014220C3014220C3014220C3014224E
:100AE0000C3014220C301422FC301422FC3014225E
:100AF0000800FF301422FF301422C3301422C33008
:100B00001422C3301422C3301422C3301422C33041
:100B100014220800C3301422C3301422C33014221C
:100B2000C3301422C3301422C3301422FF301422E5
:100B3000FF3014220800FF301422FF301422C0308E
:100B40001422C0301422C0301422C0301422FF30CE
:100B50001422FF3014220800FC301422FC3014222E
:100B60000C3014220C3014220C3014220C301422BD
:100B7000FC301422FC3014220800FF301422FF3015
:100B80001422C3301422C3301422C3301422C330C1
:100B90001422FF301422FF30142208003E301422A9
:100BA0005130142249301422453014223E30312E67
:100BB0001322423014227F3014224030142200309D
:100BC000312E423014226130142251301422493027
:100BD00014224630312E2130142241301422453067
:100BE00014224B3014223130312E1830142214309C
:100BF0001422123014227F3014221030312E27306C
:100C00001422453014224530142245301422393044
:100C1000312E3C3014224A301422493014224930FB
:100C200014223030312E0130142271301422093058
:100C30001422053014220330312E3630142249306C
:100C4000142249301422493014223630312E063015
:100C500014224930142249301422293014221E3023
:100C6000312E1422132208008C3018224030182212
:0A0C70001322132213220301312E78
:02400E00063F6B
:084200000500B800D80002001F
:00000001FF
